:0300000002085F94
:080003000220038E828F83228C
:08000B0002200BAE82AF83223C
:08001300022013742D01760098
:08001B0002201B1176017400A4
:080023000220231116017400F4
:03002B0002202B85
:10002E00216A0176016A216721792186018D01D12C
:10003E0021BA219A0208F5020B1401800201A702CF
:10004E000A5D020A63020AA102082102079E020744
:10005E00C00207F70209DC214D0207DE3098FDC20F
:10006E0098E59922117474203099FDC299F5992260
:10007E001180C0E0740D1176740A1176D0E022C2A0
:10008E00D51162319AB41B03D3E422B40D05D2D537
:10009E00C3E422FA314D40E9CA11761162319AB4A5
:1000AE001B0280E4B40D03EAC322B4080411768067
:1000BE00D0B4150280F7FB314D40E0CB1176EAC487
:1000CE004BC3227A007B007C04C2D51162319AB4F4
:1000DE001B07D3E4F583F58222B408028003B47FB4
:1000EE000CBC040280E51176313C0C80DEB40D10A0
:1000FE008B838A82BC0407E4F583F582D2D5C322B2
:10010E00FD314D40C6CD120076EDC0E0312BD0E072
:10011E002AFAE43BFBDCB4C38A828B8322EBC45401
:10012E00F0FBEAC4540F4BFBEAC454F0FA22EAC4C3
:10013E00540FFAEBC454F04AFAEBC4540FFB2224CA
:10014E00D0501424F64004240AC32224F950082463
:10015E00FA40042410C322D3223169C4C0E0540FE4
:10016E002490D43440D41176D0E022C0E0E583311F
:10017E0067E5823167D0E022C0E0E493A3600AA273
:10018E00E7547F1176400280F1D0E022B461004046
:10019E0007B47B00500224E0227800C0E0E49360B4
:1001AE0008A2E7084003A380F4D0E022C0E0C330E9
:1001BE009808E599B41B01D3C298D0E022900DB5F2
:1001CE001145EF3167EE316731861162B43A045151
:1001DE00B880EA319A75F0CBC0F075F001C0F0F539
:1001EE00F0901000F1F75024758204E493B4FE15DC
:1001FE000582E493B5F00E1174758220318611805C
:10020E00758240E4730583E583B4F8D8E5F0B43F16
:10021E0007900F1D1145A1C7B44D07900F2511452D
:10022E0081B8B45207900F2A1145A12FB4440790FC
:10023E000F2E1145419BB45507900F311145C13C0E
:10024E00B44E07900F341145E12EB44A07900F3883
:10025E001145810DB44807900F3E11458141B445BB
:10026E0007900F4A11458182B44307900F4F1145F5
:10027E00E10AB45A0B74016012900F531145E13E1E
:10028E00B44908900F4411450207640180900E4F47
:10029E0011459104116AB41B028078B43A028010A1
:1002AE00314D40F07906713380EA745E1176910417
:1002BE00790071337C007152F8742E11767152F5FB
:1002CE00837152F5827152B40102802D7022E86062
:1002DE00147152FA79017133EA120821E43402F9E9
:1002EE007133A3D8E97152EC60AA7904713380A4FA
:1002FE00E860F27152D8FC80ECE860047152D8F3D9
:10030E007152EC70E5712A900E6E114530987A118B
:10031E006A8076712A900E661145806D780079009C
:10032E00D9FED8FA22E95407232410F907E7700200
:10033E00090722D3878209878309E5827005E58341
:10034E007001C322116A319AB41B06D0E0D0E0804E
:10035E00C2B43A0A79057133D0E0D0E041C2314DD2
:10036E0050067907713380DCFA116A319AB41B0298
:10037E0080D9B43A0280DD314D5006790771338051
:10038E00E8CAC44AFA2CFCEA22EEC0E0EFC0E090C4
:10039E000E75114579107E7E7F0E91007E847F0E44
:1003AE0091007E897F0E91007A0571414009DAFA3B
:1003BE00900EC511458025900E94114579167E98A4
:1003CE007F0E71F27EA97F0E71F27EB17F0E71F2F9
:1003DE007EB77F0E71F27EBC7F0E71F2D0E0FFD041
:1003EE00E0FE0180714150091174120AA11106112B
:1003FE004522714180F27810760008B820FA2290DA
:10040E000DF7114511063179900DC5114511D12009
:10041E00D5065002E105110E1180900ED311451133
:10042E0006E4F5D0F5F07807F6D8FD758108C0E042
:10043E00C0E0737A10117E11063179743A111E7B69
:10044E00101106E493A331671174DBF711727B1060
:10045E001106E493A3547FB47F01E424E04001E449
:10046E0024201176DBEC1180D1C1110E31BA40027D
:10047E00DAC50180900E39114511063179743A11A1
:10048E001E74281176110EE4933167900E121145E9
:10049E00118D20D510400E11061208211180110663
:1004AE00A3110E8189900E440145900E01114578DD
:1004BE00151174D8FC1145758310F1F740020180B7
:1004CE001172758220318675822031A77421C398EE
:1004DE00F874201176D8FC75820031797806742074
:1004EE001176D8FC758204E493AA83B4FE05900FAE
:1004FE000B8018B4FD05900F128010B42305900FD9
:10050E000F8008B4F90280EE900F1911458A8311FD
:10051E008074F7B5830281CC0583E583B4F89B81A3
:10052E00CC117E7AFF90100015830583E583B4F815
:10053E00028021F1F7501D758204E4934403F460A8
:10054E00E911720A74412A111E1126758220318614
:10055E001180A138BAFF05900DCE0145900DC01146
:10056E004574411176111674412A1176900DC511FC
:10057E00451162B41B020180FB741FC39AEB40024B
:10058E00319A1176FB1180EB24BF50D0FBEAC39B4E
:10059E0040CA0B90100015830583E583B4F80280E2
:1005AE0017F1F75013758204E4934403F460E9DB0A
:1005BE00E71180758240812F22900EF311457C3F0A
:1005CE00900F20D1317C4DD1317C52D1317C44D130
:1005DE00317C55D1317C4ED1317C4AD1317C48D1E0
:1005EE00317C49D1317C45D1317C43D131740160AC
:1005FE00047C5AD131900F011145901000F1F75043
:10060E0020758204E493B4FE1111720582E49311F5
:10061E00761126758220318611800583E583B4F824
:10062E00DC01801172EC1176112611450180D1D3B7
:10063E00900EDD1145EB3167EA31671145ED3167FB
:10064E00EC316711808D838C82A3AC82AD83900DCB
:10065E00ED1145116AB41B02E10311808A828B836E
:10066E00ECC39582FAED95837009EA603254F0700E
:10067E000280027A10743A1176EA31673179E58395
:10068E0025822AFBE43167E49331672BFBA3DAF76B
:10069E00EBF40431671180D1C131BA50C380567466
:1006AE003A1176E431673167316704316774FF318F
:1006BE0067017EE8C0E07814E58C04000070FBD87A
:1006CE00F7D0E0F822117E900E1B114511D140217A
:1006DE0020D51EC083C0821180900E25114511D1E8
:1006EE00AD83AC82D0E0FAD0E0FB400520D502010C
:1006FE0080D0E0D0E01180900DAD0145D1D3900EA9
:10070E002F11451162319AB459EB117E8B838A8277
:10071E00E4120821EDB58305ECB5820122A380F029
:10072E00900DE4114511D140CE20D5CB110E017E96
:10073E00117E900F531145742C111E900E2F1145E2
:10074E001162319AB459AE117E1207C0900F5850F3
:10075E0003900F5F0145118078001180B88002016F
:10076E0080E83167743A11761174E6316708E854FF
:10077E000F70F580E5C0F0E493F5F0E493B5F0F971
:10078E00D0F02290DA4E74E2F090A5B1741DF022F2
:10079E00C8C0E0C082C083F19190DA4E7460F0D090
:1007AE0083D082E8F0F183E493C3686001D3D0E094
:1007BE00C82290DA4E7404F1DE908000E493F47057
:1007CE000DA37400B582F574F8B583F0C322D3225D
:1007DE00C0E0C082C083F19190DA4E7440F0F19186
:1007EE00D083D082D0E0F0E183758200E493B4A58B
:1007FE0017A3E493B4E511A3E493B4E00BA3E4933D
:10080E00B4A505758200D32274F7B58302C3220501
:10081E008380D6C0E0C0F0F5F074016010E583B4BB
:10082E00F70280225007B48002801B5019E5F0F0C9
:10083E00E493C395F06009E0C395F06003D38001A3
:10084E00C3D0F0D0E022E5F012079ED0F0D0E02227
:10085E0032E4F5A8F5B875D000115E115EF4F5809E
:10086E00F590F5A0F5B075813079C87AF9DAFED930
:10087E00FA7401601374B5600F78FAA2B579C8D90D
:10088E00FE4005D8F61207C075F0F911C811F575BE
:10089E00F0FD11C87818120080D8FB780F74201262
:1008AE000076D8FB900D76120B14900D8F120B1450
:1008BE001204B87E007F200201CB9010001207F7C1
:1008CE005024758204E493B5F015C0F0C08374E92A
:1008DE00C0E07408C0E0758240E473D083D0F005A8
:1008EE0083E583B4F8D72274007014E57B637A55E0
:1008FE006379CC63781DB57A08B57905B578022190
:10090E00BB758780759842758911E4F588F58AF56F
:10091E008CF58BF58D78C8791E30B0E5D9FBD8F7FC
:10092E0020B0FD20B0FA20B0F720B0F420B0F130A6
:10093E00B0FDD28E208FCA20B0FA208FC430B0FA0C
:10094E00208FBE20B0FAD28C208FB630B0FAC28E75
:10095E00C28C208FACE58B33F5F0E58D3340A2A22F
:10096E00F73400F404609AF58D758BFF758921D2EA
:10097E009CD28EE58DF404F978FFD8FED9FA309822
:10098E0011C298E599547F24F6600724056003028E
:10099E00090FE58A33F8E58C33F940F3E833F5F0C7
:1009AE00E933A2F7340060E7F404B58DE2F57BF588
:1009BE007AF579F578637A556379CC63781DF58D80
:1009CE00F58B758921758780759852D28E22309855
:1009DE000612006AB41B5112006AB41B4B514A2016
:1009EE009803741B2212006AB45B44514A3098DE9D
:1009FE0012006AB44103740B22B44203740A22B487
:100A0E004303741522B44403740822B435028007DC
:100A1E00B4360280028018C0E0514A30980B1200A2
:100A2E006AB47E09D0E024E422D0E080A1D0E05167
:100A3E004A30989A12006AB41BF580A1EAC0E07A97
:100A4E0014E58C2098050470FADAF6D0E0FA22C08C
:100A5E00F0C0E08013C0F0C0E030E70C742D12003F
:100A6E0076D0E0C0E0F4240175F06484D2D560073E
:100A7E00C2D52430120076E5F075F00A8430D50226
:100A8E0060052430120076E5F02430120076D0E0B6
:100A9E00D0F022C0E0E8C0E0C2D5AA82AB837C10C1
:100AAE007D2751FF60072430120076D2D57CE87D79
:100ABE000351FF700330D5072430120076D2D57C57
:100ACE00647D0051FF700330D5072430120076D2BA
:100ADE00D5EAABF075F00A84700330D505243012D8
:100AEE000076E5F08BF02430120076D0E0F8D0E0FE
:100AFE0022780008C3EA9CFAEB9DFB50F618EA2C0C
:100B0E00FAEB3DFBE822C0E0E8C0E0E9C0E0ECC053
:100B1E00E0D2D1D2D5E493A3602520E72E547FB442
:100B2E000D07120080D2D180ECB41F04C2D580E52F
:100B3E00B40E051200808007C2D112007680D6D086
:100B4E00E0FCD0E0F9D0E0F8D0E022547FF820D1DC
:100B5E0003120074C2D1C082C083900BCE7C00E819
:100B6E006007F971BD70FCD9FA71BD603CB40F120B
:100B7E0071BD0483801E68667767796278766B71C3
:100B8E006A7A0483800E657461726E69736F6C7518
:100B9E006D706463A2D592E5D2D5B81402C2E5B8E1
:100BAE000C02C2E512007680C0D083D0826123E4AD
:100BBE0093BC00057CFF540F227C00A3C4540F226B
:100BCE008290E82386054CF844B3B0B1485FF0112B
:100BDE007FA0157F1C2ED1405A50F103BFBA0C2FA7
:100BEE0096018D3F95380D6F5F1207710E562F4887
:100BFE003B6258201F7670322440B840E1618F016D
:100C0E00340BCA89D3C0A3B9588004F80285602575
:100C1E0091F092731F107F12549310444807D126FF
:100C2E00564FD0F66472E0B83BD5F0164F56306F83
:100C3E0048025FA8201F017630D5602541A42C60A4
:100C4E00056F013F261F30078E1DF06399F042B8E5
:100C5E00201F2330027AD1602FF0F6058F931A50A1
:100C6E0028F082046FA30D3F1F514023013E054320
:100C7E00017A01176493302A088C243099B0F31945
:100C8E0060254135098ECB191230051F311D041414
:100C9E004F761204AB279056012FA8D5F0AA262026
:100CAE005F1CF0F361FE0141730127C1C0848FD632
:100CBE00018770564F19701FA8D99076021743FE00
:100CCE0001C1840B157F028B14308F63396F19F0BD
:100CDE0011C9106D023F91097A41D0BA0C1D395FCE
:100CEE0007F2111720416B3509F775120BA7CC4887
:100CFE00023F6412A00C27E39FC01477701140715D
:100D0E0021C0682541F0627FD1D021E16258B0F355
:100D1E00051F733077B16F19E01943E0582FF6A411
:100D2E0014D02303FE31F5143099F8033F64225199
:100D3E006025412FE30156279309FE11FE79BA6013
:100D4E007542EA6258A0E51F534FD1C0A309425322
:100D5E00F71204621B30F505F7690C351B70822FF4
:100D6E002F144F51C064250057656C636F6D6580FD
:100D7E0094322076322E312C2062791FF81FFE0D10
:100D8E000E202053656594322E444F432C94322E00
:100D9E00455155A494322E484452B4D58D2E0E2072
:100DAE001F9E1FA0210D0E9432204C6F633A00201F
:100DBE003EA086CA822800292C958C80C83A200035
:100DCE001F9782C373C7A6832CBA204A554D5080F5
:100DDE0086A172820D0E0D0D1F8783813A20001F92
:100DEE00E4FB206B65793A20000D0D1F888083810E
:100DFE002028000D0D1F821FFD001F8120202020A6
:100E0E00201FC90E29201F871FB23A200046697283
:100E1E0073741F813A20004C6173741F813A202035
:100E2E00001FB9A120737572653F000D0D1F9C9AAE
:100E3E00922C8C80C80E20201F9CC12C8E81F70D09
:100E4E000E0D0D1F9F206173636969F9961F9884BB
:100E5E00892C958C80A00D0E0D1F8AA065640D0E39
:100E6E000D1F8AC1640D0E53756D6D6172793A0E48
:100E7E0020C67391640E208B91640E208B207772A6
:100E8E00697474656E0E1F9B3A0E208B20756E6111
:100E9E00626C65802077726974650E2020626164D1
:100EAE00F5730E20859F96C60E2085849D0E208597
:100EBE00206E6F6E849D0E1F979B20646574656314
:100ECE007465640D0E0D866E696E67823A0D0E0D99
:100EDE000D53656E64696E671F988489AC2020007F
:100EEE0020802020000D0D5374616E646172641FAA
:100EFE009E730E1FDA1FF465641F9E730E1F9A9E5B
:100F0E00001F82001F8F1FE21FAA003F3F3F001FDE
:100F1E00D7001F8ED7D1001FD18273001F8682008B
:100F2E001F8A001F93001F8781001F888083810006
:100F3E001F84DB9A83001F84DBC083001F9C9A9260
:100F4E00001FED83001FCB9990001F9990CB640D6D
:060F5E000E1F859B0D0E25
:10100000A5E5E0A5FE4C0000000000000000000087
:10101000000000000000000000000000FFFFFFFFD4
:081020004C69737400020048E2
:1010400011257D14C2D1114CDDFC0125EFF5835132
:101050004FEEF582514FE493FAA3E493FBA3E4939C
:10106000FCEA5408700FEA035478F8EA54074890F1
:1010700016C8938008EAC4540F901362935403F87F
:101080002EFEEF3400FF743A512A719D20D121EADF
:10109000514F719DB80104790B8011EB514F719D37
:1010A000B8020479088005EC514F7906719DD9FC8E
:1010B000EA54087010901748EA035478F8EA540785
:1010C0004893F980099017C8EAC4540F93F9901E09
:1010D000FE7808C374204007E99309A2E7547F51C2
:1010E0002AD8F1741BC0E07411C0E0EA5408700FF4
:1010F000EA035478F8EA5407489016C8938008EA3F
:10110000C4540F9013629354FC03031490111D23D5
:101110002582F582E43583F583E4730125412D4171
:101120003C21812172414841044152415821A22170
:10113000D7415E4169416D4108411021AA218321B7
:101140007441714177417D413E411C418121DF4124
:101150001441C54185418B41914195419B41A94134
:10116000AF41B541BB410C41BF41CB41D741E74104
:10117000ED2231F67440512A7452512AEA54014149
:101180004531F6EB20E703EB414F9012F5E493A3D2
:1011900060F5F8C39B7003020038E493A330E7FACC
:1011A00080EB511031F8742F512AEB547823C4F896
:1011B000EB54806014901372E893901F933582F57E
:1011C000825002058331978005E82420514F742E08
:1011D000512AEB5407414531F6318331F8ECFBEBF2
:1011E0002EF582EB20E703E48002E4F43FF583026E
:1011F00000367440412A5108742C512A7420412A27
:101200007423412A318331F87441412A31AA31F8DB
:101210007443412A31F25108742B512A7444512AE3
:101220007450512A7454512A7452020030EF54F809
:10123000F8EAC403540748514FEB414F31F674525A
:10124000512AEA540702002E510831F85100EB02EE
:1012500000343183ECFB414A511031F821AA510886
:1012600031F85100EB514F21DB513E416031744167
:101270006051087442412A513E31F821DF31832107
:10128000DB31AA21DB513E31F84108513E31F821D2
:1012900083513E414A318331F8413EEBC0E0ECFBE3
:1012A000318331F8D0E0FB2183318331F82174316F
:1012B0007431F84108317431F821833174414A5155
:1012C0001C31F85100EB514FEC414F31F631F251E6
:1012D00008742B512A411C31F631F25108742B51FC
:1012E0002A7450512A411031F631F2411C31F25129
:1012F0001C31F84108E04143C38153D0824450CCB3
:10130000834450C88050B09050B1A050B2B050B398
:1013100099534255C6CD5448B2C85432434FCECCEF
:10132000544CB2CB5243415032C8CA52434150325E
:10133000CC8C5448B08A544CB08D5448B18B544C2A
:10134000B1F0C2D05053D7A849C5B849D089544D3F
:101350004FC48854434FCE9853434FCE8750434F8A
:10136000CE00595909090909097A7E0976330952CB
:101370000971000206080C0E101214161B1E202301
:101380002425F8F0E493C398227950E58DF404F80D
:10139000D8FED9F722514F743A412A514F74204157
:0113A0002A22
:10140000A5E5E0A5FE53000000000000000000007C
:10141000000000000000000000000000FFFFFFFFD0
:0C14200053696E676C652D537465700095
:1014400030B306901D85020045900013E49324FEFE
:101450006005901DA88146A393F8E4A393F58288C4
:101460008374027182700EA3741471827007A37466
:10147000EF71826011A882A983901DB59146E95150
:101480004FE8514F0125E5B85404F5B8901D689117
:1014900046EF514FEE514F901D52914612003C20A5
:1014A000D50D5007901D7131970125AE82AF83C2D3
:1014B0008A901DC49146901EBC3197E4758108C086
:1014C000E0C0E08E828F83F5D0F8F9FAFBFCFDFED8
:1014D000FFF5F0757CDD757D14D2AAD2AF737189EA
:1014E000D0E0F9D0E0F8D082D083D0D0D0E032C0C4
:1014F000E0C0D0C083C082E8C0E0E9C0E07189D21A
:1015000099719D719DE58124FBF8E6719BE5F07171
:101510009B08E62354015145719D08E6514F08E6AA
:10152000719B719D08E6719508E67195EA7195EBDE
:101530007195EC7195ED7195EE7195EF719B719DC3
:10154000E824F8719B719D719DE57C8E7CFEE57DA4
:101550008F7DFFEAC0E0EBC0E0ECC0E0D2D1114CDF
:10156000D0E0FCD0E0FBD0E0FAAF7DAE7CE581249A
:10157000F9F8E6F57C08E6F57D120062120040B449
:101580000D0281DEB4200281DEB43F07901E35914A
:1015900046A179B45113901EB53197C2AA718975CD
:1015A000080075090075810932B44802A1CDB45212
:1015B00002A1FDB45302C167B44102C1AAB42E070F
:1015C000901EBC3197A179A179743D412A901E03E8
:1015D0003197E47195719DA88118E6719B08E651D9
:1015E0004F7802790EA1ECE871957910719DE65162
:1015F0004F08D9F81125B880EE1125A17990134430
:101600003197B1C9E58124FCF8E6719B901348A895
:10161000A8D16090134BA8B8D16090134EA889D17F
:1016200060901353A888D160901358A898D1609007
:10163000135DA887D1607454512A7430512AB1C9FE
:10164000E58C514FE58A514F719D7454512A743184
:10165000512AB1C9E58D514FE58B514F1125A17923
:101660003197B1C9E8619B7817719DD8FC901DEB4B
:101670003197E58124F9F8E68E7CFE08E68F7DFF40
:10168000EAC0E0EBC0E0ECC0E0D2D1114CD0E0FC0D
:10169000D0E0FBD0E0FAE58124F9F8EEAE7CF57CF1
:1016A000F608EFAF7DF57DF6A179E58124FBF89092
:1016B0001E25319712003A400820D505F61125A1C4
:1016C00079901D713197A179AD066F393946494935
:1016D00063066F39394649496306AD39160E111153
:1016E0006306AD39160E111166061A1F160E11117A
:1016F00066061A1F160E111166061A1F160E111114
:1017000066062269161F9292660622A14D8386867E
:101710009B06969D160E11112606225D4DAD8E8EEE
:101720002606423D2F2B37374606423D390E111112
:101730004606423D39571111A5061111390E1111F6
:10174000A9068989391A89895A0E48732B2B2B2BA4
:1017500030004375212121212E0E676E06060606F4
:1017600038006A700A0A0A0A330E5D5D5D5D5D5DD0
:101770003B00121212121212410E8F8F8F8F8F8F19
:101780003E005D354C4C4C4C7C0E124F244C4C4C66
:101790004C004C4F808080805D0E4C2B57924C4CFF
:1017A00012001C1C15151515630E191984888888DC
:1017B000600078781F278B8B530E5353194C4C4C79
:1017C000530053531C4C4C4C2B21060A5D128F4C7A
:0817D0004C804C1588274C4C9D
:10180000A5E5E0A5FE450000000000000000000086
:10181000000000000000000000000000FFFFFFFFCC
:101820004D656D6F727920456469746F722028561A
:06183000543130302900A4
:101840007C0051C6ECC2E3FC1200623119B41B02E9
:10185000618DB40B024124B40A02414BB408024129
:1018600066B415024195B40C0451C60144B411028A
:10187000618DB4030FEC54FEFC71CF901D36B14660
:1018800051E10144B4040FEC4401FC71CF901D3BC5
:10189000B14651E10144B4070221ECB4050221E054
:1018A000B406022159B4010FEC30E198D2E2FC9168
:1018B00054916471210144B4180FEC30E186C2E206
:1018C000FC9154916471210144B419024141B41A4C
:1018D000024146F5F0EC20E102014430E210E5F06F
:1018E0007198B5F0F48F838E821200564195E5F021
:1018F00012004012006540E1F88F838E82EC20E3F5
:101900000AE8FDECD2E3FC71210148EDC454F02853
:10191000120056ECC2E3FC4195C0E0EC20E106C2A7
:10192000E3FCD0E02230E3F9D0E0C0E01200401246
:10193000006550EED0E0C0E0B41B0EECC2E3FC71D9
:1019400021D0E0D0E0D0E001448F838E82ED120000
:1019500056ECC2E3FC712180C9EC540270020144D0
:101960009154ECC0E09019C2B14C12003C404820A8
:10197000D545A882A9839019D2B14612003C4037C0
:1019800020D534AC82AD839019DBB14C12003A40C3
:101990002620D523FAECFEEDFFD0E0FC8882898377
:1019A000EA120056EEB5820CEFB5830891549164AB
:1019B00051E10144A380E9D0E0FC9154916471218C
:1019C000014446696C6C1F833B2046697273743A0C
:1019D000200020204C6173743A200020A83A200097
:1019E0009154EC6402FC9164712101449154901A69
:1019F0001DB14CECC0E012003CD0E0FC401320D5FF
:101A000010AE82AF8371CF741471D5916451E1012E
:101A10004471CF741471D59164712101441F831FE7
:101A2000813A2000714DEEC39410FEEF9400FFEE5A
:101A3000F454F06008740171DD7169014451E101F1
:101A4000441F51E101440F51E10144714DEE241056
:101A5000FEEF3400FFEE54F06008740171D5716937
:101A6000014451E10144714D740371E5EEC39401E9
:101A7000FEEF9400FFEE44F0F4600471690144EE5F
:101A8000F454F0600C743071ED740171DD71690112
:101A90004451E10144714D740371ED8E828F83A333
:101AA000AE82AF83EE540F600471690144EE54F0CE
:101AB000600C743071E5740171D57169014451E1B4
:101AC00001447420A140901CFCB146913BB1499166
:101AD00018B1499132B149741071D59132B149911F
:101AE0006471CF740271D57582008F837810B1490B
:101AF000120036743AB140AA82AB8351C271AAB1C6
:101B000043A3E582540F70F38A828B8351C251C282
:101B100051C271AA7198B140A3E582540F70F3D8F5
:101B2000CD71CFEEC4540F240371D5EE540F243879
:101B300071ED71F571B37198B1409101EE540F23BD
:101B4000F4243471E571F571B3B1438101EE540FA2
:101B500023F4243171ED71B37198B140EE540F2329
:101B6000F4243471E571B3A143EE540F23F424310E
:101B700071ED71B3719871F5B1409101EE540F237D
:101B8000F4243471E571B371F5B1438101EE54F081
:101B9000C4F4241371D5A149547FB47F0374202267
:101BA000C3942050027400242022EC20E003E4932C
:101BB00022E022C083C0828F838E82EC20E30D203E
:101BC000E004E4938001E0D082D08322ED80F8919C
:101BD0000B7448A140910BB14F7442A140910BB1DD
:101BE0004F7441A140910BB14F7444A140910BB18E
:101BF0004F7443A140901BFAA1461B5B303B376DED
:101C000000901C06A1461B5B306D00C0E0741BB148
:101C100040745BB140D0E022901D04B14678005181
:101C2000C2742BB140E812002E08B810F2901D0AC1
:101C3000A1467848742DB140D8FA22EC20E00590F6
:101C40001D368003901D3BB146780851C2D8FC90E8
:101C50001D1EA14C71CF741471D57A4851C2DAFCA3
:101C6000744861E5EC30E112901CBC20E203901C4A
:101C7000D7B146901CF2B1468005901CB4B1469095
:101C80001C84A14620205E473D476F746F20205E74
:101C9000433D436F646520205E443D446174612090
:101CA000205E4C3D52656472617720205E513D514B
:101CB000756974005E452D45646974005E413D1B85
:101CC0005B303B376D41534349491B5B306D2020EE
:101CD0005E583D486578005E413D41534349492087
:101CE000205E583D1B5B303B376D4865781B5B3091
:101CF0006D0020205E463D46696C6C001B5B481BF6
:101D00005B324A00414444523A0020202041534370
:101D10004949204551554956494C414E54003830A7
:101D200035311F9A1F831FD86F722C1FF81FFE2C8E
:101D3000203139393600434F444500444154410075
:101D4000020030020034020038020048020045025E
:101D50000050292C206F72203C4553433E20746F65
:101D600020657869743A20000D1F888083812028BF
:101D70000020436F6D6D616E642041626F72746507
:101D8000642E0D0A000DA1C520636F6E6E6563742D
:101D900020494E5431202870696E20313329206C3F
:101DA0006F7780BACFCC0D009432B3C7AE812030AC
:101DB0003031330D001FB8B3FFA520766563746F13
:101DC00072AE20000D4E6F77866E696E67A6CFCC1F
:101DD000206D6F64653A20203C5245543E3DCC2C2A
:101DE000203F3D2048656C700D0D00536B6970708D
:101DF000696E6720496E737472756374696F6E2DB6
:101E00003E20000D0A4C6F633A2020496E74205228
:101E1000414D204D656D6F727920436F6E74656E14
:101E200074730D0A004E6577204163632056616C20
:101E300075653A20000D1FCF1FCC1F9E3A0D3C52F6
:101E400045543E2086D4F60D203C53503E2086D487
:101E5000F60D20273F272020FF8ED70D20272E2785
:101E60002020FFC4FD730D202752272020FF207360
:101E700070656369616C2066756E6374696F6EC4AA
:101E8000730D20274827202084DBC0920D20275384
:101E9000272020FCD4F60D202741272020F0A22067
:101EA0004163632076616C75650D202751272020E2
:101EB000C8CFCC0D0E517569740D0A002020414326
:101EC000432042204320445054522020523020527C
:101ED0003120523220523320523420523520523693
:101EE000205237202053502020204164647220204B
:101EF000496E737472756374696F6E0D0A004143A5
:101F0000414CCC004144C400414444C3414A4DD0FB
:101F1000414ECC434A4EC5434CD24350CC44C144BD
:101F200045C34449D6444A4EDA494EC34AC24A429E
:101F3000C34AC34A4DD04A4EC24A4EC34A4EDA4AF9
:101F4000DA4C43414CCC4C4A4DD04D4FD64D4F56B8
:101F5000C34D4F56D84D55CC4E4FD04F52CC504F0D
:101F6000D0505553C85245D4524554C952CC524C06
:101F7000C352D25252C3534554C2534A4DD0535503
:101F800042C2535741D05843C8584348C45852CC12
:101F90003F3FBF50B054434FCE50B153434FCE504C
:101FA000B249C550B349D043B05432434FCE5053D9
:091FB000D744B84143C3FDC2FE51
:00000001FF
